:020000040000FA
:0A0000000000000097EF01F0AAD104
:08001800F7D1076A066EFF0E26
:100020000626072200D0D8A01200030E056EE60EA9
:1000300002D8F5D7056AFE0F046EE86A055AD8A003
:1000400012000000040600D0F8D7800E1C1A1B50C6
:10005000175C206E11E2206C17501BC017F01B6E4E
:1000600018501CC018F01C6E19501DC019F01D6EE0
:100070001A501EC01AF01E6E1A0E206074D01B5249
:1000800072E01F6A1850226E1C18236E188E1C8E88
:10009000080E205E08E31EC01FF01DC01EF01CC02D
:1000A0001DF01C6AF5D7202607E0D8901C321D32BF
:1000B0001E321F32202EF9D723AE33D01E501A5EC7
:1000C0001D50195A1C50185A07E2D880000E1A56B3
:1000D00019561856800E221A1F6C04E01A06000EDC
:1000E000195A185A040E206E18660DD019C018F04F
:1000F0001AC019F01FC01AF01F6A080E175E29E314
:10010000202EF2D726D018BE08D0D8901F361A3627
:1001100019361836172EF7D71CD01FAE22D01F6AFB
:100120000FD01E501A261D5019221C50182206E30B
:10013000183219321A321F32174A0DD01FAE11D0A1
:100140001A3E0FD0193E0DD0183E0BD0D8801A9011
:10015000EFD7176A02D0218217681A6A196A800ECF
:10016000186E22AE189E1A5012001850166E1C18E7
:10017000236E1750D8A41B503AE017267E0E03E3D7
:10018000175E03E336D0175E31E31AC014F019C0CE
:1001900015F0168E1C8E1A6A196A186A180E226ECD
:1001A00016321532143206E31E501A261D5019223B
:1001B0001C501822183219321A32222EF1D718BECA
:1001C00007D01A3619361836175210E017061634AB
:1001D00016E31A3E14D0193E12D0183E10D0D88023
:1001E000183219321A32173E0AD003D02184176A06
:1001F00002D0218217681A6A196A800E186E23AE1F
:10020000189E1A50120017C022F018501AC018F089
:100210001A6E1A3622321A32216A1A36223602E34E
:100220002184217E06E12180226A1A6A196A186AED
:100230000BD0222803E0D8801A3206D0D8901A3288
:1002400002E1218201D0218621B604D021A20FD063
:1002500021B407D07F0E1A6EFF0E196E186E176E3E
:1002600023D0800E1A6E01D01A6A000EF6D721B084
:10027000FBD7176A9F0E2260EBD77E0E2264F4D75D
:100280009E0E225C07E0D8901A32193218321732CB
:10029000222AF6D721A408D0D880000E1756185667
:1002A00019561A561AAEE0D717501200176E186A70
:1002B000196A1A6A239E0AD0239E1AAE07D0D880E4
:1002C000000E1756185619561A56238E960E226E81
:1002D0001A5209E0080E222618C017F019C018F0AB
:1002E0001AC019F011D019520FE1080E225E1850F1
:1002F00007E1080E225E175002E11A5010D0176A6B
:10030000196E17C018F0176A19BE06D0D8901736A4
:10031000183619362206F8D723AE199E225017C078
:100320001AF0176E195018C019F0186E1200400E0E
:10033000216E4F0EAF6E240EAC6E900EAB6E0001B0
:100340000F0EC16E070EB46EC69AC00E926EE00E0E
:10035000936EC00E946E956AE80E966E6CD0F2A401
:1003600003D0F294817A11009EAA19D0060EAB1424
:1003700012E1E2CF7DF0E1CF7CF07E2A11EE00F0B9
:100380007E50E126000EE222AECFE7FF7DC0E2FF05
:100390007CC0E1FF1100AE50AE50AB98AB881100AD
:1003A0007E507F5C14E07F2AEACF05F0E9CF04F0AD
:1003B00001EE00F07F50E926000EEA22EF50046EB5
:1003C00005C0EAFF04C0E9FFD880120004D0E86845
:1003D000046ED8A0120012007E6A7F6A9D8A9F8AEE
:1003E000F28EF28C12009D9A01EE00F0010EF46E76
:1003F000F36AF306000EF45AEE6AF450F310F9E1D2
:100400007E6A7F6A9D8A1200F29EE0CFE3F4D8CF25
:10041000E4F4E8CFE5F4F28E0001A192F29EE3C489
:10042000E0FFE4C4D8FFE5C4E8FFF28E10009EA808
:10043000FED7AD6E1200939A8A8A0A0E0DEC00F078
:10044000939A8A9A95928C92929289929294899494
:10045000929689969290899092988998929A899A80
:1004600096908D9096928D9296948D9493988A986A
:1004700093968A9693948A9493928A9293908A9070
:10048000959E8C9E959C8C9C959A8C9A95988C9810
:10049000949A8B9A94988B9895968C9695948C9424
:1004A00094908B9094928B9294948B9495908C9042
:1004B00094968B965A6A596A586A576A566A556A68
:1004C00000EEB2F0300EEE68E82EFDD78B6BA66B17
:1004D000A76BA86BA96BAA6BAB6BAC6BAD6BAE6B70
:1004E000AF6BB06BB16B8D6B8C6B8F6B8E6B916BDD
:1004F000906B936B926B956B946B976B966B996B00
:10050000986B9B6B9A6B9D6B9C6B9F6B9E6BA16BAF
:10051000A06BA36BA26BA56BA46B5C6A5B6A5E6A43
:100520005D6A606A5F6A626A616A646A636A666A6F
:10053000656A686A676A6A6A696A6C6A6B6A6E6A1F
:100540006D6A706A6F6AE26B47DF4DDFCD6AF294C5
:10055000F28A870ED56EB16AA192A082D08EA29245
:10056000B10EB16ED5EC0DF0D7EC0FF0752AE86A3C
:1005700075B2010F76B0010806E17670712A000E9F
:100580007222732274220CDF246EC50E245C06E3F3
:10059000FE0E245C01E2256AC6EF07F024AE29D0E6
:1005A000256A840E245C05E124C025F02668816953
:1005B0001ED0940E245C05E124C025F0276828682D
:1005C00016D0A40E245C05E124C025F0826983695D
:1005D0000ED0B40E245C05E124C025F08469856941
:1005E00006D0C40E245C03E124C025F08669C4EF64
:1005F00007F0255204E1C6EF07F0C4EF07F0840EC0
:10060000255CD8A4A9D0262803E124C026F0A0D0D8
:1006100024C081F0300E265C08E15590579059B007
:1006200002D0899401D0899290D0310E265C08E1E5
:100630005592579259B002D0899001D0899685D0B1
:10064000320E265C08E15594579459B402D089982B
:1006500001D08D927AD0330E265C08E155965796DC
:1006600059B602D08D9001D08D926FD0340E265C99
:1006700008E15598579859B802D08D9401D08A98BE
:1006800064D0350E265C08E1559A579A59BA02D0C3
:100690008A9601D08A9459D0360E265C08E1559C82
:1006A000579C59BC02D08A9201D08A904ED0370E06
:1006B000265C08E1559E579E59BE02D08C9E01D003
:1006C0008C9C43D0380E265C08E1569058905AB066
:1006D00002D08C9A01D08C9838D0390E265C08E173
:1006E000569258925AB202D08B9A01D08B982DD044
:1006F0003A0E265C08E1569458945AB402D08C966F
:1007000001D08C9422D03B0E265C08E15696589678
:100710005AB602D08B9001D08B9217D07A0E265CFD
:1007200005E18B942668C6EF07F00FD07B0E265CA0
:1007300005E18C902668C6EF07F007D07C0E265C9A
:1007400004E18B962668C6EF07F02668C4EF07F031
:10075000C6EF07F0C4EF07F0940E255CD8A49EEF17
:1007600007F0272804E124C027F09CEF07F024C0FD
:1007700028F02852D8A49FD0300E275C08E155906D
:10078000579059B002D0899401D0899290D0310EFF
:10079000275C08E15592579259B002D0899001D058
:1007A000899685D0320E275C08E15594579459B448
:1007B00002D0899801D08D927AD0330E275C08E15F
:1007C0005596579659B602D08D9001D08D926FD024
:1007D000340E275C08E15598579859B802D08D948B
:1007E00001D08A9864D0350E275C08E1559A579A53
:1007F00059BA02D08A9601D08A9459D0360E275C15
:1008000008E1559C579C59BC02D08A9201D08A902D
:100810004ED0370E275C08E1559E579E59BE02D038
:100820008C9E01D08C9C43D0380E275C08E15690FA
:1008300058905AB002D08C9A01D08C9838D0390E8A
:10084000275C08E1569258925AB202D08B9A01D096
:100850008B982DD03A0E275C08E1569458945AB4E0
:1008600002D08C9601D08C9422D03B0E275C08E1FC
:10087000569658965AB602D08B9001D08B9217D0CC
:100880007A0E275C05E18B942668C6EF07F00FD03F
:100890007B0E275C05E18C902668C6EF07F007D039
:1008A0007C0E275C04E18B962668C6EF07F0C4EF48
:1008B00007F09CEF07F0300E275CD8A440D059B069
:1008C00003D08994898202D0899289845970558095
:1008D00002EEE3F0D8902834E926000EEA22EECFAB
:1008E000A4F0EFCFA5F0A4517124006EA5517220A1
:1008F000016E000E7320026E000E7420036E03C0A2
:10090000B5F002C0B4F001C0B3F000C0B2F0A6531D
:1009100013E0578003EEE3F0D890A635E926000EE9
:10092000EA22EECF00F0EFCF01F0A451005C8C6F13
:10093000A55101588D6F01D057909AEF07F0310EF5
:10094000275CD8A440D059B203D08990898602D0C0
:10095000899689805972558202EEE3F0D890283446
:10096000E926000EEA22EECF5BF0EFCF5CF05B50A1
:100970007124006E5C507220016E000E7320026EB6
:10098000000E7420036E03C0B9F002C0B8F001C0BD
:10099000B7F000C0B6F0A75313E0578203EEE3F0C0
:1009A000D890A735E926000EEA22EECF00F0EFCF6F
:1009B00001F05B50005C8E6F5C5001588F6F01D06E
:1009C00057929AEF07F0320E275CD8A440D059B462
:1009D00003D08998898A02D0899A89885974558464
:1009E00002EEE3F0D8902834E926000EEA22EECF9A
:1009F0005DF0EFCF5EF05D507124006E5E507220AE
:100A0000016E000E7320026E000E7420036E03C090
:100A1000BDF002C0BCF001C0BBF000C0BAF0A853EA
:100A200013E0578403EEE3F0D890A835E926000ED2
:100A3000EA22EECF00F0EFCF01F05D50005C906F46
:100A40005E500158916F01D057949AEF07F0330E22
:100A5000275CD8A440D059B603D08D908D8202D0A7
:100A60008D928D805976558602EEE3F0D890283429
:100A7000E926000EEA22EECF5FF0EFCF60F05F5084
:100A80007124006E60507220016E000E7320026EA1
:100A9000000E7420036E03C0C1F002C0C0F001C09C
:100AA000BFF000C0BEF0A95313E0578603EEE3F099
:100AB000D890A935E926000EEA22EECF00F0EFCF5C
:100AC00001F05F50005C926F60500158936F01D04D
:100AD00057969AEF07F0340E275CD8A43FD059B848
:100AE00003D08D948A8802D08A988D84597855884D
:100AF00002EEE3F0D8902834E926000EEA22EECF89
:100B000061F0EFCF62F061507124006E625072208C
:100B1000016E000E7320026E000E7420036E03C07F
:100B2000C5F002C0C4F001C0C3F000C0C2F0AA53B7
:100B300013E0578803EEE3F0D890AA35E926000EBB
:100B4000EA22EECF00F0EFCF01F06150005C946F2D
:100B500062500158956F01D05798ECD1350E275C43
:100B6000D8A43FD059BA03D08A968A8402D08A94F6
:100B70008A86597A558A02EEE3F0D8902834E9261D
:100B8000000EEA22EECF63F0EFCF64F063507124E1
:100B9000006E64507220016E000E7320026E000E13
:100BA0007420036E03C0C9F002C0C8F001C0C7F0D2
:100BB00000C0C6F0AB5313E0578A03EEE3F0D890C1
:100BC000AB35E926000EEA22EECF00F0EFCF01F0C0
:100BD0006350005C966F64500158976F01D0579A2C
:100BE000A9D1360E275CD8A43FD059BC03D08A9235
:100BF0008A8002D08A908A82597C558C02EEE3F07A
:100C0000D8902834E926000EEA22EECF65F0EFCF27
:100C100066F065507124006E66507220016E000E01
:100C20007320026E000E7420036E03C0CDF002C06C
:100C3000CCF001C0CBF000C0CAF0AC5313E0578C2D
:100C400003EEE3F0D890AC35E926000EEA22EECFB1
:100C500000F0EFCF01F06550005C986F66500158CE
:100C6000996F01D0579C66D1370E275CD8A43FD02E
:100C700059BE03D08C9E8C8C02D08C9C8C8E597E5D
:100C8000558E02EEE3F0D8902834E926000EEA22D1
:100C9000EECF67F0EFCF68F067507124006E6850B8
:100CA0007220016E000E7320026E000E7420036E1F
:100CB00003C0D1F002C0D0F001C0CFF000C0CEF030
:100CC000AD5313E0578E03EEE3F0D890AD35E9262F
:100CD000000EEA22EECF00F0EFCF01F06750005C8B
:100CE0009A6F685001589B6F01D0579E23D1380EE0
:100CF000275CD8A43FD05AB003D08C9A8C8802D0FD
:100D00008C988C8A5A70568002EEE3F0D890283482
:100D1000E926000EEA22EECF69F0EFCF6AF06950C3
:100D20007124006E6A507220016E000E7320026EF4
:100D3000000E7420036E03C0D5F002C0D4F001C0D1
:100D4000D3F000C0D2F0AE5313E0588003EEE3F0CE
:100D5000D890AE35E926000EEA22EECF00F0EFCFB4
:100D600001F06950005C9C6F6A5001589D6F01D082
:100D70005890E0D0390E275CD8A43FD05AB203D0A7
:100D80008B9A8B8802D08B988B8A5A72568202EE8D
:100D9000E3F0D8902834E926000EEA22EECF6BF07B
:100DA000EFCF6CF06B507124006E6C507220016EAE
:100DB000000E7320026E000E7420036E03C0D9F083
:100DC00002C0D8F001C0D7F000C0D6F0AF5313E096
:100DD000588203EEE3F0D890AF35E926000EEA2200
:100DE000EECF00F0EFCF01F06B50005C9E6F6C50C7
:100DF00001589F6F01D058929DD03A0E275CD8A41D
:100E00003FD05AB403D08C968C8402D08C948C86BC
:100E10005A74568402EEE3F0D8902834E926000E86
:100E2000EA22EECF6DF0EFCF6EF06D507124006EC0
:100E30006E507220016E000E7320026E000E742040
:100E4000036E03C0DDF002C0DCF001C0DBF000C0C7
:100E5000DAF0B05313E0588403EEE3F0D890B035E5
:100E6000E926000EEA22EECF00F0EFCF01F06D5040
:100E7000005CA06F6E500158A16F01D058945AD0F9
:100E80003B0E275CD8A43FD05AB603D08B908B8200
:100E900002D08B928B805A76568602EEE3F0D89081
:100EA0002834E926000EEA22EECF6FF0EFCF70F083
:100EB0006F507124006E70507220016E000E73200E
:100EC000026E000E7420036E03C0E1F002C0E0F079
:100ED00001C0DFF000C0DEF0B15313E0588603EE2E
:100EE000E3F0D890B135E926000EEA22EECF00F00B
:100EF000EFCF01F06F50005CA26F70500158A36FEC
:100F000001D0589617D07A0E275C04E18B842768AD
:100F10003DD010D07B0E275C04E18C80276836D052
:100F200009D07C0E275C04E18B8627682FD002D085
:100F300027682CD0276828D029D026D0A40E255C7D
:100F40000BE1822903E124C082F004D024C083F0A5
:100F500069EC0BF01BD018D0B40E255C0BE1842992
:100F600003E124C084F004D024C085F093EC0CF09D
:100F70000DD00AD0C40E255C07E1862904E124C007
:100F800086F07EEC0CF002D02FEC0BF00C0E7B5CAC
:100F9000D8B027EF0BF07750715C785072587950C9
:100FA00073587A507458D8A016EF0BF07A8E7B5293
:100FB000D8A442D059B002D0899401D0899257B0B8
:100FC00006D05590B569B469B369B26933D055A0FC
:100FD00016D08C517124006E8D517220016E000E5E
:100FE0007320026E000E7420036E03C0B5F002C0C1
:100FF000B4F001C0B3F000C0B2F055901BD059B0AE
:1010000002D0898201D089845970A4517124006E64
:10101000A5517220016E000E7320026E000E742026
:10102000036E03C0B5F002C0B4F001C0B3F000C05D
:10103000B2F0558015EF0BF0010E7B5CD8A442D0C6
:1010400059B202D0899001D0899657B206D05592F4
:10105000B969B869B769B66933D055A216D08E514F
:101060007124006E8F517220016E000E7320026E8B
:10107000000E7420036E03C0B9F002C0B8F001C0C6
:10108000B7F000C0B6F055921BD059B202D0898695
:1010900001D0898059725B507124006E5C507220BF
:1010A000016E000E7320026E000E7420036E03C0EA
:1010B000B9F002C0B8F001C0B7F000C0B6F0558278
:1010C00015EF0BF0020E7B5CD8A442D059B402D0CD
:1010D000899801D0899A57B406D05594BD69BC69E6
:1010E000BB69BA6933D055A416D090517124006EF3
:1010F00091517220016E000E7320026E000E74205A
:10110000036E03C0BDF002C0BCF001C0BBF000C064
:10111000BAF055941BD059B402D0898A01D089887D
:1011200059745D507124006E5E507220016E000E85
:101130007320026E000E7420036E03C0BDF002C067
:10114000BCF001C0BBF000C0BAF0558415EF0BF045
:10115000030E7B5CD8A442D059B602D08D9001D04A
:101160008D9257B606D05596C169C069BF69BE69F0
:1011700033D055A616D092517124006E935172202F
:10118000016E000E7320026E000E7420036E03C009
:10119000C1F002C0C0F001C0BFF000C0BEF0559663
:1011A0001BD059B602D08D8201D08D8059765F5008
:1011B0007124006E60507220016E000E7320026E6A
:1011C000000E7420036E03C0C1F002C0C0F001C065
:1011D000BFF000C0BEF0558615EF0BF0040E7B5C2F
:1011E000D8A441D059B802D08D9401D08A9857B86C
:1011F00006D05598C569C469C369C26933D055A87A
:1012000016D094517124006E95517220016E000E1B
:101210007320026E000E7420036E03C0C5F002C07E
:10122000C4F001C0C3F000C0C2F055981BD059B83B
:1012300002D08A8801D08D84597861507124006E63
:1012400062507220016E000E7320026E000E742038
:10125000036E03C0C5F002C0C4F001C0C3F000C0FB
:10126000C2F05588E2D1050E7B5CD8A441D059BAB2
:1012700002D08A9601D08A9457BA06D0559AC96985
:10128000C869C769C66933D055AA16D0965171246A
:10129000006E97517220016E000E7320026E000ED8
:1012A0007420036E03C0C9F002C0C8F001C0C7F0CB
:1012B00000C0C6F0559A1BD059BA02D08A8401D01A
:1012C0008A86597A63507124006E64507220016ED0
:1012D000000E7320026E000E7420036E03C0C9F06E
:1012E00002C0C8F001C0C7F000C0C6F0558A9DD149
:1012F000060E7B5CD8A441D059BC02D08A9201D0A2
:101300008A9057BC06D0559CCD69CC69CB69CA6917
:1013100033D055AC16D098517124006E995172207B
:10132000016E000E7320026E000E7420036E03C067
:10133000CDF002C0CCF001C0CBF000C0CAF0559C8B
:101340001BD059BC02D08A8001D08A82597C65505A
:101350007124006E66507220016E000E7320026EC2
:10136000000E7420036E03C0CDF002C0CCF001C0AB
:10137000CBF000C0CAF0558C58D1070E7B5CD8A4C6
:1013800041D059BE02D08C9E01D08C9C57BE06D055
:10139000559ED169D069CF69CE6933D055AE16D08C
:1013A0009A517124006E9B517220016E000E7320C1
:1013B000026E000E7420036E03C0D1F002C0D0F0A4
:1013C00001C0CFF000C0CEF0559E1BD059BE02D058
:1013D0008C8C01D08C8E597E67507124006E6850C1
:1013E0007220016E000E7320026E000E7420036ED8
:1013F00003C0D1F002C0D0F001C0CFF000C0CEF0E9
:10140000558E13D1080E7B5CD8A441D05AB002D0BF
:101410008C9A01D08C9858B006D05690D569D46972
:10142000D369D26933D056A016D09C517124006E76
:101430009D517220016E000E7320026E000E74200A
:10144000036E03C0D5F002C0D4F001C0D3F000C0D9
:10145000D2F056901BD05AB002D08C8801D08C8A22
:101460005A7069507124006E6A507220016E000E2D
:101470007320026E000E7420036E03C0D5F002C00C
:10148000D4F001C0D3F000C0D2F05680CED0090E07
:101490007B5CD8A441D05AB202D08B9A01D08B98F1
:1014A00058B206D05692D969D869D769D66933D06F
:1014B00056A216D09E517124006E9F517220016E6B
:1014C000000E7320026E000E7420036E03C0D9F06C
:1014D00002C0D8F001C0D7F000C0D6F056921BD0A1
:1014E0005AB202D08B8801D08B8A5A726B50712409
:1014F000006E6C507220016E000E7320026E000EA2
:101500007420036E03C0D9F002C0D8F001C0D7F038
:1015100000C0D6F0568289D00A0E7B5CD8A441D098
:101520005AB402D08C9601D08C9458B406D05694FC
:10153000DD69DC69DB69DA6933D056A416D0A051C5
:101540007124006EA1517220016E000E7320026E94
:10155000000E7420036E03C0DDF002C0DCF001C099
:10156000DBF000C0DAF056941BD05AB402D08C8461
:1015700001D08C865A746D507124006E6E507220AA
:10158000016E000E7320026E000E7420036E03C005
:10159000DDF002C0DCF001C0DBF000C0DAF0568400
:1015A00044D00B0E7B5CD8A440D05AB602D08B90AE
:1015B00001D08B9258B606D05696E169E069DF6992
:1015C000DE6933D056A616D0A2517124006EA35105
:1015D0007220016E000E7320026E000E7420036EE6
:1015E00003C0E1F002C0E0F001C0DFF000C0DEF0B7
:1015F00056961BD05AB602D08B8201D08B805A7679
:101600006F507124006E70507220016E000E7320B6
:10161000026E000E7420036E03C0E1F002C0E0F021
:1016200001C0DFF000C0DEF0568619D874AE0ED0CF
:10163000746A736A726A716A566A556A586A576A36
:1016400000EEB2F0300EEE68E82EFDD706D074AE94
:1016500004D0746A736A726A716AB6EF02F07B68CA
:101660007A8E806B0C0E805D33E2D8908035E96E07
:10167000EA6AEA36E936EA36B20EE926000EEA22CE
:10168000EFCF00F0ECCF01F0ECCF02F0ECCF03F0A5
:101690007750005C78500158795002587A500358BE
:1016A00015E2D8908035E96EEA6AEA36E936EA361C
:1016B000B20EE926000EEA22EFCF77F0ECCF78F0F9
:1016C000ECCF79F0ECCF7AF080C07BF0802BCAE3CE
:1016D0001200300E825D14E183C0A6F0A6530CE028
:1016E00003EEE3F0D890A635E926000EEA22EECF0D
:1016F0008CF0EFCF8DF003D08D6B8C6B5790FCD0BE
:10170000310E825D14E183C0A7F0A7530CE003EE15
:10171000E3F0D890A735E926000EEA22EECF8EF04E
:10172000EFCF8FF003D08F6B8E6B5792E5D0320ED8
:10173000825D14E183C0A8F0A8530CE003EEE3F04F
:10174000D890A835E926000EEA22EECF90F0EFCF30
:1017500091F003D0916B906B5794CED0330E825D95
:1017600014E183C0A9F0A9530CE003EEE3F0D89094
:10177000A935E926000EEA22EECF92F0EFCF93F0E2
:1017800003D0936B926B5796B7D0340E825D14E101
:1017900083C0AAF0AA530CE003EEE3F0D890AA3578
:1017A000E926000EEA22EECF94F0EFCF95F003D0B9
:1017B000956B946B5798A0D0350E825D14E183C071
:1017C000ABF0AB530CE003EEE3F0D890AB35E92679
:1017D000000EEA22EECF96F0EFCF97F003D0976B92
:1017E000966B579A89D0360E825D14E183C0ACF0B7
:1017F000AC530CE003EEE3F0D890AC35E926000ED4
:10180000EA22EECF98F0EFCF99F003D0996B986B66
:10181000579C72D0370E825D14E183C0ADF0AD539A
:101820000CE003EEE3F0D890AD35E926000EEA2295
:10183000EECF9AF0EFCF9BF003D09B6B9A6B579E45
:101840005BD0380E825D14E183C0AEF0AE530CE085
:1018500003EEE3F0D890AE35E926000EEA22EECF93
:101860009CF0EFCF9DF003D09D6B9C6B589044D0C3
:10187000390E825D14E183C0AFF0AF530CE003EE8C
:10188000E3F0D890AF35E926000EEA22EECF9EF0C5
:10189000EFCF9FF003D09F6B9E6B58922DD03A0EE6
:1018A000825D14E183C0B0F0B0530CE003EEE3F0CE
:1018B000D890B035E926000EEA22EECFA0F0EFCFA7
:1018C000A1F003D0A16BA06B589416D03B0E825DA3
:1018D00013E183C0B1F0B1530CE003EEE3F0D89014
:1018E000B135E926000EEA22EECFA2F0EFCFA3F049
:1018F00003D0A36BA26B589682691200865307E14E
:10190000E25304E0D7EC0FF086C0E2F00AD07A0E82
:10191000865D07E17A0EE25D04E04EEC10F086C0D1
:10192000E2F0866912001E0E845DD8A4C6D08553ED
:1019300027E1586A576A8D6B8C6BA66B8F6B8E6B29
:10194000A76B916B906BA86B936B926BA96B956B6C
:10195000946BAA6B976B966BAB6B996B986BAC6B3C
:101960009B6B9A6BAD6B9D6B9C6BAE6B9F6B9E6B19
:10197000AF6BA16BA06BB06BA36BA26BB16B9CD078
:1019800085C0A6F003EEE3F0D8908535E926000E79
:10199000EA22EECF8CF0EFCF8DF085C0A7F003EEFA
:1019A000E3F0D8908535E926000EEA22EECF8EF0DE
:1019B000EFCF8FF085C0A8F003EEE3F0D890853527
:1019C000E926000EEA22EECF90F0EFCF91F085C02D
:1019D000A9F003EEE3F0D8908535E926000EEA225F
:1019E000EECF92F0EFCF93F085C0AAF003EEE3F0D4
:1019F000D8908535E926000EEA22EECF94F0EFCF9D
:101A000095F085C0ABF003EEE3F0D8908535E9267C
:101A1000000EEA22EECF96F0EFCF97F085C0ACF043
:101A200003EEE3F0D8908535E926000EEA22EECFEA
:101A300098F0EFCF99F085C0ADF003EEE3F0D890C9
:101A40008535E926000EEA22EECF9AF0EFCF9BF023
:101A500085C0AEF003EEE3F0D8908535E926000EA0
:101A6000EA22EECF9CF0EFCF9DF085C0AFF003EE01
:101A7000E3F0D8908535E926000EEA22EECF9EF0FD
:101A8000EFCF9FF085C0B0F003EEE3F0D89085353E
:101A9000E926000EEA22EECFA0F0EFCFA1F085C03C
:101AA000B1F003EEE3F0D8908535E926000EEA2286
:101AB000EECFA2F0EFCFA3F00FD0420E845D08E18D
:101AC000855303E18B910AD802D08B818C8204D09C
:101AD0007B0E845DD8B449D8846912008C92566A12
:101AE000556A586A576A89928996899A8D928A9816
:101AF0008A948A908C9C8C988B988C948B928994E5
:101B0000899089988D908D948A968A928C9E8C9AD1
:101B10008B9A8C968B908B948C908B968D6B8C6B18
:101B2000A66B8F6B8E6BA76B916B906BA86B936B97
:101B3000926BA96B956B946BAA6B976B966BAB6B67
:101B4000996B986BAC6B9B6B9A6BAD6B9D6B9C6B45
:101B5000AE6B9F6B9E6BAF6BA16BA06BB06BA36BFF
:101B6000A26BB16BE26BD7EF0FF0566A556A586AF9
:101B7000576A89928996899A8D928A988A948A90CE
:101B80008C9C8C988B988C948B9289948990899852
:101B90008D908D948A968A928C9E8C9A8B9A8C9634
:101BA0008B908B948C908B9612000301E469E3690F
:101BB000AA0EE66F480EE56FA40EE86FCC0EE76F35
:101BC000A20EEA6F1E0EE96F9F0EEC6F7C0EEB6F9C
:101BD0009C0EEE6FE50EED6F9A0EF06F590EEF6FE3
:101BE000970EF26FD70EF16F950EF46F600EF36FD4
:101BF000920EF66FF30EF56F900EF86FF76F8E0E74
:101C0000FA6F370EF96F8B0EFC6FE80EFB6F890EC3
:101C1000FE6FA20EFD6F870E0401006F660E0301BA
:101C2000FF6F850E0401026F330E016F830E046F88
:101C3000090E036F800E066FE90E056F7E0E086FAA
:101C4000D10E076F7C0E0A6FC10E096F7A0E0C6FF2
:101C5000BB0E0B6F780E0E6FBC0E0D6F760E106FF5
:101C6000C60E0F6F740E126FD90E116F720E146FB5
:101C7000F30E136F710E166F150E156F6F0E186F32
:101C80003F0E176F6D0E1A6F700E196F6B0E1C6F73
:101C9000A90E1B6F690E1E6FEA0E1D6F680E206F76
:101CA000310E1F6F660E226F800E216F640E246F3F
:101CB000D60E236F630E266F330E256F610E286FCD
:101CC000960E276F600E2A6F010E296F5E0E2C6F25
:101CD000720E2B6F5C0E2E6FE90E2D6F5B0E306F48
:101CE000670E2F6F590E326FEB0E316F580E346F37
:101CF000750E336F570E366F050E356F550E386FF4
:101D00009B0E376F540E3A6F370E396F520E3C6F81
:101D1000D90E3B6F510E3E6F810E3D6F500E406FDE
:101D20002E0E3F6F4E0E426FE10E416F4D0E446F0F
:101D3000990E436F4C0E466F560E456F4B0E486F13
:101D4000190E476F490E4A6FE00E496F480E4C6FEF
:101D5000AD0E4B6F470E4E6F7F0E4D6F460E506FA0
:101D6000560E4F6F450E526F320E516F440E546F28
:101D7000120E536F420E566FF70E556F410E586F8D
:101D8000E00E576F400E5A6FCF0E596F3F0E5C6FCB
:101D9000C10E5B6F3E0E5E6FB80E5D6F3D0E606FE5
:101DA000B30E5F6F3C0E626FB30E616F3B0E646FDC
:101DB000B60E636F3A0E666FBE0E656F390E686FB2
:101DC000CA0E676F380E6A6FDA0E696F370E6C6F66
:101DD000ED0E6B6F370E6E6F050E6D6F360E706FFA
:101DE000200E6F6F350E726F3F0E716F340E746F71
:101DF000620E736F330E766F880E756F320E786FCA
:101E0000B20E776F310E7A6FDF0E796F310E7C6F05
:101E1000100E7B6F300E7E6F440E7D6F2F0E806F25
:101E20007B0E7F6F2E0E826FB60E816F2D0E846F2C
:101E3000F30E836F2D0E866F340E856F2C0E886F18
:101E4000780E876F2B0E8A6FBF0E896F2B0E8C6FEB
:101E50000A0E8B6F2A0E8E6F570E8D6F290E906FA4
:101E6000A70E8F6F280E926FF90E916F280E946F48
:101E70004F0E936F270E966FA80E956F270E986FD3
:101E8000030E976F260E9A6F610E996F250E9C6F49
:101E9000C10E9B6F250E9E6F240E9D6FA06F8A0E44
:101EA0009F6F230EA26FF20EA16F230EA46F5C0E24
:101EB000A36F220EA66FC90EA56F220EA86F390E52
:101EC000A76F210EAA6FAA0EA96F210EAC6F1E0E6E
:101ED000AB6F200EAE6F950EAD6F200EB06F0D0E76
:101EE000AF6F1F0EB26F880EB16F1F0EB46F050E6D
:101EF000B36F1E0EB66F840EB56F1E0EB86F050E53
:101F0000B76F1D0EBA6F880EB96F1D0EBC6F0D0E28
:101F1000BB6F1C0EBE6F950EBD6F1C0EC06F1E0EEC
:101F2000BF6F1B0EC26FA90EC16F1B0EC46F360EA2
:101F3000C36F1A0EC66FC50EC56F1A0EC86F560E48
:101F4000C76F190ECA6FE80EC96F190ECC6F7C0EE1
:101F5000CB6F190ECE6F120ECD6F180ED06FAA0E6A
:101F6000CF6F180ED26F440ED16F170ED46FDF0EE5
:101F7000D36F170ED66F7B0ED56F170ED86F1A0E54
:101F8000D76F160EDA6FBA0ED96F160EDC6F5B0EB6
:101F9000DB6F150EDE6FFE0EDD6F150EE06FA30E0C
:101FA000DF6F150EE26F490EE16F00011200010EA6
:101FB000806F800E805DD8B070D00B6A800E0A6E84
:101FC000180E096E880E086E1F0E0F6E850E0E6EAF
:101FD000370E0D6E820E0C6E805156EC01F01AC059
:101FE00013F019C012F018C011F017C010F01E6ADB
:101FF0001D6A1C6A7F0E1B6E13C01AF012C019F006
:1020000011C018F010C017F025EC00F01AC013F042
:1020100019C012F018C011F017C010F00FC01EF058
:102020000EC01DF00DC01CF00CC01BF013C01AF048
:1020300012C019F011C018F010C017F0B5EC00F084
:102040001AC00FF019C00EF018C00DF017C00CF038
:102050000BC01EF00AC01DF009C01CF008C01BF028
:102060000FC01AF00EC019F00DC018F00CC017F018
:1020700027EC00F003EC01F0006E18C001F002EE56
:10208000E3F0D8908035E926000EEA2200C0EEFF8A
:1020900001C0EFFF802BD8A08CD71200010E806FFB
:1020A000800E805DD8B06FD00B6A0A6A520E096E3E
:1020B000850E086E520E0F6EB80E0E6E130E0D6E5C
:1020C000840E0C6E805156EC01F01AC013F019C04A
:1020D00012F018C011F017C010F01E6A1D6A1C6AB9
:1020E0007F0E1B6E13C01AF012C019F011C018F049
:1020F00010C017F025EC00F01AC013F019C012F050
:1021000018C011F017C010F00FC01EF00EC01DF067
:102110000DC01CF00CC01BF013C01AF012C019F057
:1021200011C018F010C017F0B5EC00F01AC00FF095
:1021300019C00EF018C00DF017C00CF00BC01EF047
:102140000AC01DF009C01CF008C01BF00FC01AF037
:102150000EC019F00DC018F00CC017F027EC00F0FD
:1021600003EC01F0006E18C001F002EEE3F0D8902D
:102170008035E926000EEA2200C0EEFF01C0EFFF25
:0A218000802BD8A08DD71200FFD7E6
:020000040030CA
:0300010006160ED2
:020005008580F4
:060008000FC00FE00F40E5
:00000001FF
